:020000040800F2
:1000000000060020E1010008D50E00088D0E000852
:10001000B50E00088D0E0008AD0E0008E3010008C3
:10002000E3010008E3010008E30100089527000848
:10003000E3010008E3010008E3010008E301000810
:10004000E3010008E3010008E3010008E301000800
:10005000E3010008E3010008313800085D380008BA
:1000600089380008B5380008E1380008E3010008C5
:10007000E3010008E3010008E3010008E3010008D0
:10008000E3010008E3010008E3010008E3010008C0
:10009000E3010008E3010008E30100080D3900084E
:1000A000E3010008E3010008E3010008E3010008A0
:1000B000A5360008E3010008E3010008E301000899
:1000C000E3010008E3010008E3010008E301000880
:1000D000E30100082D0F0008E3010008E301000818
:1000E00075390008E3010008E3010008E301000896
:1000F000E3010008E3010008E3010008E301000850
:10010000E3010008E3010008E3010008E30100083F
:10011000E3010008E3010008E3010008E30100082F
:10012000E3010008E3010008E3010008E30100081F
:10013000E3010008E3010008E3010008E30100080F
:10014000E3010008E3010008E3010008CD2E0008E8
:10015000E3010008E3010008E3010008E3010008EF
:10016000E3010008E3010008E3010008E3010008DF
:10017000E3010008E3010008E3010008E3010008CF
:10018000E3010008E3010008E3010008E3010008BF
:10019000E3010008E3010008E3010008E3010008AF
:1001A000E3010008E3010008E3010008E30100089F
:1001B000E3010008E3010008E3010008E30100088F
:1001C000E3010008E3010008E3010008E30100087F
:1001D000E3010008E3010008E3010008E30100086F
:1001E00002E000F000F8FEE772B63A4880F30888B3
:1001F000394880F3098839484EF60851CEF200019B
:10020000086040F20000CCF200004EF63471CEF2ED
:1002100000010860BFF34F8FBFF36F8F40F2000003
:10022000C0F2F0004EF68851CEF200010860BFF334
:100230004F8FBFF36F8F4FF00000E1EE100A4EF6C4
:100240003C71CEF200010860062080F31488BFF3F1
:100250006F8F02F01FFB02F0FBFA03F087F94FF0FB
:1002600055301F491B4A91423CBF41F8040BFAE745
:100270001C49194A91423CBF41F8040BFAE71A495C
:100280001A4A1B4B9A423EBF51F8040B42F8040B2A
:10029000F8E700201749184A91423CBF41F8040B87
:1002A000FAE702F0D9FA03F0B5F9144C144DAC4258
:1002B00003DA54F8041B8847F9E700F041F8114CC1
:1002C000114DAC4203DA54F8041B8847F9E702F0F9
:1002D000C1BA000000060020002200200000000833
:1002E0000000002000060020F03D00080022002051
:1002F0004C2200205022002030300020E001000875
:10030000E0010008E0010008E00100082DE9F04FDD
:100310002DED108AC1F80CD0C3689D46BDEC108A43
:10032000BDE8F08F002383F311882846A047002002
:1003300001F03CFEFEE701F0B7FD00DFFEE7000044
:1003400038B502F0F7F9054602F01AFA0446D8B9B2
:100350000F4B9D421AD001339D4218BF044641F213
:10036000883504BF01240025002002F0EDF90CB10E
:1003700000F076F800F028FD00F0BAFB284600F007
:10038000C3F800F06DF8F9E70025EDE70546EBE767
:10039000010007B008B500F077FBA0F12003584238
:1003A000584108BD07B541F21203022101A8ADF87A
:1003B000043000F087FB03B05DF804FB38B5202360
:1003C00083F311881748C3680BB101F075FE164A14
:1003D000144800234FF47A7101F032FE002383F3B6
:1003E0001188124C236813B12368013B23606368B2
:1003F00013B16368013B63600D4D2B7833B96368BB
:100400007BB9022000F052FC322363602B78032B6F
:1004100007D163682BB9022000F048FC4FF47A73CF
:10042000636038BD50220020BD0300086C2300200B
:1004300064220020084B187003280CD8DFE800F075
:1004400008050208022000F021BC022000F00EBCCA
:10045000024B00225A607047642200206C23002067
:10046000244B254A10B51C461968013140D004338D
:100470009342F9D16268214B9A4239D9204B9B684B
:1004800003F1006303F580339A4231D2002000F07B
:1004900049FB0220FFF7CEFF1A4B1A6C00221A64A8
:1004A000196E1A66196E596C5A64596E5A665A6EEC
:1004B0005A6942F080025A615A6922F080025A61F8
:1004C0005A691A6942F000521A611A6922F0005200
:1004D0001A611B6972B64FF0E0232021C3F8084D62
:1004E000D4E9003281F311889D4683F308881047D0
:1004F00010BD00BF0000010820000108FFFF000838
:1005000000220020003802402DE9F04F93B0AA4BA2
:1005100000902022FF210AA89D6800F0FFFBA74A57
:100520001378A3B9A6480121C3601170202383F377
:100530001188C3680BB101F0BFFDA24AA048002397
:100540004FF47A7101F07CFD002383F31188009B46
:1005500013B19D4B009A1A609C4A009C1378032BA0
:100560001EBF00231370984A4FF0000A18BF536053
:10057000D3465646D146012000F088FB24B1924B69
:100580001B68002B00F01182002000F07DFA039020
:10059000039B002BF2DB012000F068FB039B213B57
:1005A000162BE8D801A252F823F000BF0906000874
:1005B00031060008C5060008770500087705000821
:1005C000770500084F0700081F09000839080008D0
:1005D0009B080008C3080008E90800087705000820
:1005E000FB080008770500086D090008A906000847
:1005F00077050008B109000815060008A9060008DB
:10060000770500089B0800080220FFF7C3FE0028BA
:1006100040F0F581009B0221BAF1000F08BF1C4693
:1006200005A841F21233ADF8143000F04BFAA2E7FE
:100630004FF47A7000F028FA071EEBDB0220FFF778
:10064000A9FE0028E6D0013F052F00F2DA81DFE89D
:1006500007F0030A0D10133605230593042105A89E
:1006600000F030FA17E054480421F9E75848042113
:10067000F6E758480421F3E74FF01C08404600F025
:1006800053FA08F104080590042105A800F01AFAAD
:10069000B8F12C0FF2D1012000FA07F747EA0B0B53
:1006A0005FFA8BFB4FF0000900F084FB26B10BF0E2
:1006B0000B030B2B08BF0024FFF774FE5BE74648D3
:1006C0000421CDE7002EA5D00BF00B030B2BA1D1FD
:1006D0000220FFF75FFE074600289BD0012000F0B4
:1006E00021FA0220FFF7A6FE00265FFA86F84046B0
:1006F00000F028FA044690B10021404600F032FA9A
:1007000001360028F1D1BA46044641F21213022103
:1007100005A8ADF814303E4600F0D4F92BE70120CF
:10072000FFF788FE2546244B9B68AB4207D9284635
:1007300000F0FAF9013040F067810435F3E7234B0C
:1007400000251D70204BBA465D603E46ACE7002E8A
:100750003FF460AF0BF00B030B2B7FF45BAF022079
:10076000FFF768FE322000F08FF9B0F10008FFF6C5
:1007700051AF18F003077FF44DAF0F4A926808EBB2
:10078000050393423FF646AFB8F5807F3FF742AF8F
:10079000124B0193B84523DD4FF47A7000F074F9E1
:1007A0000390039A002AFFF635AF019B039A03F8E2
:1007B000012B0137EDE700BF002200206823002055
:1007C00050220020BD0300086C230020642200207A
:1007D00004220020082200200C2200206822002091
:1007E000C820FFF7D7FD074600283FF413AF1F2DA1
:1007F00011D8C5F1200242450AAB25F0030028BFFD
:10080000424683490192184400F062FA019A8048F6
:10081000FF2100F083FA4FEAA8037D490193C8F352
:100820008702284600F082FA064600283FF46DAFA2
:10083000019B05EB830537E70220FFF7ABFD00289E
:100840003FF4E8AE00F0BAF900283FF4E3AE002729
:10085000B846704B9B68BB4218D91F2F11D80A9B12
:1008600001330ED027F0030312AA134453F8203C9F
:1008700005934046042205A900F02EFB043780466C
:10088000E7E7384600F050F90590F2E7CDF814801C
:10089000042105A800F016F906E70023642104A846
:1008A000049300F005F900287FF4B4AE0220FFF7AE
:1008B00071FD00283FF4AEAE049800F067F9059092
:1008C000E6E70023642104A8049300F0F1F800286F
:1008D0007FF4A0AE0220FFF75DFD00283FF49AAE42
:1008E000049800F063F9EAE70220FFF753FD0028BF
:1008F0003FF490AE00F072F9E1E70220FFF74AFD05
:1009000000283FF487AE05A9142000F06DF90421FA
:100910000746049004A800F0D5F83946B9E732201C
:1009200000F0B2F8071EFFF675AEBB077FF472AE9B
:10093000384A926807EB090393423FF66BAE0220F8
:10094000FFF728FD00283FF465AE27F003074F446A
:10095000B9453FF4A9AE484600F0E6F804210590F9
:1009600005A800F0AFF809F10409F1E74FF47A7037
:10097000FFF710FD00283FF44DAE00F01FF90028EE
:1009800044D00A9B01330BD008220AA9002000F0B2
:10099000CDF900283AD02022FF210AA800F0BEF9A4
:1009A000FFF700FD1C4801F007FB13B0BDE8F08F16
:1009B000002E3FF42FAE0BF00B030B2B7FF42AAE6F
:1009C0000023642105A8059300F072F8074600286B
:1009D0007FF420AE0220FFF7DDFC804600283FF4C4
:1009E00019AEFFF7DFFC41F2883001F0E5FA059817
:1009F00000F02AFA464600F0DDF93C46BBE5064623
:100A000052E64FF0000905E6BA467EE637467CE638
:100A10006822002000220020A08601002DE9F84F66
:100A20004FF47A73DFF85880DFF8589006460D4689
:100A300002FB03F7002498F900305A1C5FFA84FA8D
:100A400001D0A34212D159F8240003682A46D3F8F2
:100A500020B031463B46D847854207D1074B01209D
:100A600083F800A0BDE8F88F0124E4E7002CFBD058
:100A70004FF4FA7001F0A0FA0020F3E7B42300204D
:100A8000102200201422002007B500230246012175
:100A90000DF107008DF80730FFF7C0FF20B19DF87A
:100AA000070003B05DF804FB4FF0FF30F9E70000EA
:100AB0000A4608B50421FFF7B1FF80F00100C0B27B
:100AC000404208BD30B4074B0A461978064B53F82C
:100AD00021402368DD69054B0146AC46204630BC09
:100AE000604700BFB423002014220020A08601002C
:100AF00070B501F011FD094E094D308000242868C1
:100B00003388834208D901F001FD2B680444013386
:100B1000B4F5803F2B60F2D370BD00BFB623002038
:100B20007423002001F0BABD00F1006000F58030B0
:100B30000068704700F10060920000F5803001F01D
:100B400039BD0000054B1A68054B1B889B1A834270
:100B500002D9104401F0DABC002070477423002051
:100B6000B623002038B5084D044629B12868204432
:100B7000BDE8384001F0EABC2868204401F0CEFC12
:100B80000028F3D038BD00BF7423002010F0030309
:100B90000AD1B0F5047F05D200F10050A0F5104055
:100BA000D0F80038184670470023FBE700F10050EA
:100BB000A0F51040D0F8100A70470000064991F8DF
:100BC000243033B10023086A81F824300822FFF76B
:100BD000B1BF0120704700BF78230020014B186887
:100BE000704700BF002004E0F0B51C4B02461868B7
:100BF0001B4BC0F30B050424000C1E88AE421BD116
:100C00005C6893F90850174B05261F88874208BF78
:100C100093F90250013E03F10403F6D1013A0A446C
:100C2000013C0B4693420ED214F9016F581C66B179
:100C300000F8016C0346F5E7013C03F10C03DCD13D
:100C4000094C3F25DFE7184605E02C2490421C7034
:100C500001D2981C5D70401AF0BD00BF002004E076
:100C6000B83A0008A43A0008783A0008022804D1EB
:100C7000054B4FF080429A6170470128FCD1024B2E
:100C80004FF00052F7E700BF00000240022804D1F5
:100C9000054B4FF480429A6170470128FCD1024B0A
:100CA0004FF40052F7E700BF00000240022805D1D0
:100CB000064A536983F48043536170470128FCD18D
:100CC000024A536983F40053F6E700BF0000024074
:100CD00010B50023934203D0CC5CC4540133F9E730
:100CE00010BD000010B5013810F9013F3BB191F97A
:100CF00000409C4203D11AB10131013AF4E71AB124
:100D000091F90020981A10BD1046FCE703460246F0
:100D1000D01A12F9011B0029FAD170470244034688
:100D2000934202D003F8011BFAE770472DE9F8431C
:100D30001F4D144695F824200746884652BBDFF81D
:100D400070909CB395F824302BB92022FF2148469F
:100D50002F62FFF7E3FF95F82400C0F10802A242DA
:100D600028BF2246D6B24146920005EB8000FFF72D
:100D7000AFFF95F82430A41B1E44F6B2082E17448A
:100D80009044E4B285F82460DBD1FFF717FF002818
:100D9000D7D108E02B6A03EB82038342CFD0FFF761
:100DA0000DFF0028CBD10020BDE8F8830120FBE730
:100DB00078230020024B1A78024B1A70704700BF4C
:100DC000B42300201022002038B5194C194D2046BC
:100DD00000F008FC2946204600F030FC2D6816483B
:100DE0006A6DD2F8043843F00203C2F8043801F007
:100DF000E3F82846114900F027FD6A6D104DD2F83E
:100E0000043828680F4923F00203C2F80438A042CE
:100E10004FF4E1330B6001D000F044FB6868A0425E
:100E200004D0BDE83840074900F03CBB38BD00BFE6
:100E3000D8270020E83B000840420F00F03B0008A4
:100E400014220020A023002070B50C4B0C4D1E78FE
:100E50000C4B55F826209A4204460DD00A4B00212F
:100E600014221846FFF75AFF0460014655F8260081
:100E7000BDE8704000F016BB70BD00BFB423002079
:100E800014220020D8270020A023002000B59BB00A
:100E9000EFF3098168226846FFF71AFFEFF3058335
:100EA000014B9B6BFEE700BF00ED00E008B5FFF7CC
:100EB000EDFF000000B59BB0EFF3098168226846A2
:100EC000FFF706FFEFF30583014B5B6BFEE700BF07
:100ED00000ED00E0FEE7000030B5094D0A44914204
:100EE0000DD011F8013B5840082340F30004013BAA
:100EF0002C4013F0FF0384EA5000F6D1EFE730BD39
:100F00002083B8ED024AD36843F0C003D360704732
:100F100000100140044B5A6810439A6858600AB1A7
:100F2000181D1047704700BFB82300202DE9F0417D
:100F30003C4ED6F85C52EF682B68DA059CB20CD5B3
:100F4000202383F311884FF40070FFF7E3FF6FF461
:100F500080732B60002383F31188202383F311888F
:100F6000DFF8C08014F02F0339D183F311883806DD
:100F700013D5210611D5202383F311882A4800F0C8
:100F8000EFF900284CDA0820FFF7C4FF4FF67F7313
:100F90003B40EB60002383F311887A0615D5630686
:100FA00013D5202383F31188D6E913239A4209D15C
:100FB000336C3BB127F040073F0410203F0CFFF794
:100FC000A9FFEF60002383F31188D6F86422D36869
:100FD0000BB110699847BDE8F04101F00FBC230741
:100FE00012D014F0080F0CBF00208020E10748BF8A
:100FF00040F02000A20748BF40F04000630748BF10
:1010000040F48070FFF786FFA4066B6805D596F85C
:1010100060124046194000F053FA2C68A4B2A1E7D0
:101020006860B7E7B8230020F023002010B5054C16
:10103000054A0021204600F013FA044BC4F85C3244
:1010400010BD00BFB8230020050F000800100140AC
:1010500038B52A4C037C002918BF0C46012B0546E5
:10106000C0F8644210D1264B98420DD1254B5A6CE2
:1010700042F010025A645A6E42F010025A660B2176
:1010800025205B6E00F046F8D5F85C221E492368E7
:101090008A424FEA530003D001F580618A422AD187
:1010A0001A490144B4F90400B1FBF3F30028BEBFB0
:1010B00023F0070003F0070343EA4003A18893608D
:1010C000E38843F040031361238943F00103536134
:1010D00041F4045343F02C03D36001F4A0510023E6
:1010E0001360B1F5806F136853680CBF7F23FF2333
:1010F00085F8603238BD0649D3E700BFE83A0008FA
:10110000B8230020003802400010014000BD010556
:1011100080DE800200F1604303F561430901C9B23A
:1011200083F80013012200F01F039A4043099B003B
:1011300003F1604303F56143C3F880211A607047EF
:10114000F8B5154682680669AA420B46816938BF20
:101150008568761AB54204460BD218462A46FFF730
:10116000B7FDA3692B44A361A3685B1BA36028465A
:10117000F8BD0CD918463246FFF7AAFDAF1BE1684F
:101180003A463044FFF7A4FDE3683B44EBE71846DA
:101190002A46FFF79DFDE368E5E700008368934278
:1011A000F7B51546044638BF8568D0E90460361A9D
:1011B000B5420BD22A46FFF78BFD63692B4463616E
:1011C000A36828465B1BA36003B0F0BD0DD932466F
:1011D0000191FFF77DFD0199E068AF1B3A4631446C
:1011E000FFF776FDE3683B44E9E72A46FFF770FD29
:1011F000E368E4E710B50A440024C361029B8460FD
:10120000C0E90000C0E90511C1600261036210BDC0
:1012100008B5D0E90532934201D1826882B982686B
:10122000013282605A1C42611970D0E904329A423C
:1012300024BFC3684361002100F0DAFE002008BD2E
:101240004FF0FF30FBE7000070B5202304460E4648
:1012500083F31188A568A5B1A368A269013BA360C7
:10126000531CA36115782269934224BFE368A361EC
:10127000E3690BB120469847002383F31188284681
:1012800007E03146204600F0A3FE0028E2DA85F3AD
:10129000118870BD2DE9F74F04460E461746984653
:1012A000D0F81C904FF0200A8AF311884FF0000B01
:1012B000154665B12A4631462046FFF741FF0346F1
:1012C00060B94146204600F083FE0028F1D000239B
:1012D00083F31188781B03B0BDE8F08FB9F1000FDC
:1012E00003D001902046C847019B8BF31188ED1A6B
:1012F0001E448AF31188DCE7C0E90511C160C361AF
:101300001144009B8260C0E90000016103627047E4
:10131000F8B504460D461646202383F31188A768C6
:10132000A7B1A368013BA36063695A1C62611D7089
:10133000D4E904329A4224BFE3686361E3690BB1E4
:1013400020469847002080F3118807E03146204668
:1013500000F03EFE0028E2DA87F31188F8BD0000B5
:10136000D0E905239A4210B501D182687AB9826822
:10137000013282605A1C82611C7803699A4224BF40
:10138000C3688361002100F033FE204610BD4FF09A
:10139000FF30FBE72DE9F74F04460E461746984607
:1013A000D0F81C904FF0200A8AF311884FF0000B00
:1013B000154665B12A4631462046FFF7EFFE034643
:1013C00060B94146204600F003FE0028F1D000231A
:1013D00083F31188781B03B0BDE8F08FB9F1000FDB
:1013E00003D001902046C847019B8BF31188ED1A6A
:1013F0001E448AF31188DCE70268436811430160E8
:1014000003B11847704700001430FFF743BF0000D6
:101410004FF0FF331430FFF73DBF00003830FFF7C7
:10142000B9BF00004FF0FF333830FFF7B3BF000003
:101430001430FFF709BF00004FF0FF311430FFF701
:1014400003BF00003830FFF763BF00004FF0FF32EA
:101450003830FFF75DBF000000207047FFF7E6BDA2
:1014600037B515460E4A026000224260C0E90222EA
:101470000122044602740B46009000F15C014FF417
:1014800080721430FFF7B6FE00942B464FF4807242
:1014900004F5AE7104F13800FFF72EFF03B030BD44
:1014A000FC3A000810B52023044683F31188FFF7A7
:1014B000CFFD02232374002383F3118810BD0000A5
:1014C00038B5C36904460D461BB904210844FFF72B
:1014D00093FF294604F11400FFF79AFE002806DA6C
:1014E000201D4FF48061BDE83840FFF785BF38BD4F
:1014F000026843681143016003B118477047000058
:1015000013B5446BD4F894341A681178042915D1B2
:10151000217C022912D11979128901238B401342AF
:101520000CD101A904F14C0001F026FFD4F8944439
:10153000019B21790246206800F0CEF902B010BD6F
:10154000143001F0A9BE00004FF0FF33143001F059
:10155000A3BE00004C3001F07BBF00004FF0FF3312
:101560004C3001F075BF0000143001F077BE000070
:101570004FF0FF31143001F071BE00004C3001F02B
:1015800047BF00004FF0FF324C3001F041BF000078
:101590000020704710B5D0F894341A6811780429E7
:1015A000044617D1017C022914D1597952890123AB
:1015B0008B4013420ED1143001F00AFE024648B1AE
:1015C000D4F894444FF4807361792068BDE81040EA
:1015D00000F070B910BD0000406BFFF7DBBF0000EA
:1015E000704700007FB5124B036000234360C0E9E1
:1015F0000233012502260F4B057404460290019325
:1016000000F18402294600964FF48073143001F0F3
:10161000BBFD094B0294CDE9006304F523724FF43E
:101620008073294604F14C0001F082FE04B070BDC5
:10163000243B0008D9150008011500080B6820227A
:1016400082F311880A7903EB820290614A790932A8
:1016500043F822008A7912B103EB820398610223D6
:101660000374C0F89414002383F3118870470000BA
:1016700038B5037F044613B190F85430ABB9201D40
:1016800001250221FFF734FF04F1140025776FF0E4
:10169000010100F0B9FC84F8545004F14C006FF0E3
:1016A0000101BDE8384000F0AFBC38BD10B50121E4
:1016B00004460430FFF71CFF0023237784F85430DE
:1016C00010BD000038B504460025143001F074FD4B
:1016D00004F14C00257701F043FE201D84F854509E
:1016E0000121FFF705FF2046BDE83840FFF752BF54
:1016F00090F8443003F06003202B07D190F8452088
:10170000212A4FF0000303D81F2A06D80020704773
:10171000222AFBD1C0E90E3303E0034A8263072289
:10172000C2630364012070471C22002037B5D0F843
:1017300094341A681178042904461AD1017C0229CC
:1017400017D11979128901238B40134211D100F16D
:101750004C05284601F0C4FE58B101A9284601F005
:101760000BFED4F89444019B21790246206800F0D6
:10177000B3F803B030BD0000F0B500EB810385B0D5
:101780009E6904460D46FEB1202383F3118804EBC5
:101790008507301D0821FFF7ABFEFB685B691B68FE
:1017A00006F14C001BB1019001F0F4FD019803A972
:1017B00001F0E2FD024648B1039B2946204600F0B5
:1017C0008BF8002383F3118805B0F0BDFB685A69DC
:1017D0001268002AF5D01B8A013B1340F1D104F1B5
:1017E0004402EAE7093138B550F82140DCB1202342
:1017F00083F31188D4F894241368527903EB82039D
:10180000DB689B695D6845B104216018FFF770FED5
:10181000294604F1140001F0E5FC2046FFF7BAFE6A
:10182000002383F3118838BD7047000001F0A8B889
:10183000012303700023C0E90133C36183620362A3
:10184000C36243620363704738B50446202383F3C1
:1018500011880025C0E90355C0E90555416001F034
:101860009FF80223237085F3118838BD70B500EB13
:10187000810305465069DA600E46144618B11022FD
:101880000021FFF74BFAA06918B110220021FFF7E1
:1018900045FA31462846BDE8704001F04BB90000DA
:1018A000826802F0011282600022C0E90422826193
:1018B00001F0CCB9F0B400EB81044789E46801255C
:1018C000A4698D403D43458123600023A26063608D
:1018D000F0BC01F0E7B90000F0B400EB8104078927
:1018E000E468012564698D403D4305812360002340
:1018F000A2606360F0BC01F061BA000070B5022321
:10190000002504460370C0E90255C0E90455C564CA
:10191000856180F8345001F0A9F863681B6823B131
:1019200029462046BDE87040184770BD037880F80E
:1019300050300523037043681B6810B504460BB193
:10194000042198470023A36010BD000090F85020A8
:10195000436802701B680BB10521184770470000EF
:1019600070B590F83430044613B1002380F8343059
:1019700004F14402204601F08BF963689B68B3B917
:1019800094F8443013F0600535D00021204601F072
:10199000DDFB0021204601F0CFFB63681B6813B11B
:1019A000062120469847062384F8343070BD20462F
:1019B00098470028E4D0B4F84A30E26B9A4288BFD6
:1019C000E36394F94430E56B002B4FF0200380F281
:1019D0000381002D00F0F280092284F8342083F383
:1019E00011880021D4E90E232046FFF775FF00235C
:1019F00083F31188DAE794F8452003F07F0343EA84
:101A0000022340F20232934200F0C58021D8B3F5A0
:101A1000807F48D00DD8012B3FD0022B00F093805F
:101A2000002BB2D104F14C02A2630222E2632364D0
:101A3000C1E7B3F5817F00F09B80B3F5407FA4D16F
:101A400094F84630012BA0D1B4F84C3043F0020397
:101A500032E0B3F5006F4DD017D8B3F5A06F31D099
:101A6000A3F5C063012B90D8636894F846205E68A4
:101A700094F84710B4F848302046B047002884D086
:101A80004368A3630368E3631AE0B3F5106F36D0CD
:101A900040F6024293427FF478AF5C4BA36302238B
:101AA000E3630023C3E794F84630012B7FF46DAF66
:101AB000B4F84C3023F00203C4E90E55A4F84C30BE
:101AC000256478E7B4F84430B3F5A06F0ED194F8EC
:101AD000463084F84E30204601F020F863681B68D9
:101AE00013B1012120469847032323700023C4E942
:101AF0000E339CE704F14F03A3630123C3E723786C
:101B0000042B10D1202383F311882046FFF7C8FE51
:101B100085F311880321636884F84F5021701B6896
:101B20000BB12046984794F84630002BDED084F85D
:101B30004F300423237063681B68002BD6D002212A
:101B400020469847D2E794F848301D0603F00F016D
:101B500020460AD501F08EF8012804D002287FF42F
:101B600014AF2B4B9AE72B4B98E701F075F8F3E78E
:101B700094F84630002B7FF408AF94F8483013F007
:101B80000F01B3D01A06204602D501F0F3FAADE7F3
:101B900001F0E6FAAAE794F84630002B7FF4F5AEA0
:101BA00094F8483013F00F01A0D01B06204602D550
:101BB00001F0CCFA9AE701F0BFFA97E7142284F813
:101BC000342083F311882B462A4629462046FFF706
:101BD00071FE85F31188E9E65DB1152284F83420A1
:101BE00083F311880021D4E90E232046FFF762FE1B
:101BF000FDE60B2284F8342083F311882B462A4615
:101C000029462046FFF768FEE3E700BF543B000883
:101C10004C3B0008503B000838B590F8343004467F
:101C2000002B3ED0063BDAB20F2A34D80F2B32D825
:101C3000DFE803F0373131082232313131313131CF
:101C400031313737C56BB0F84A309D4214D2C36882
:101C50001B8AB5FBF3F203FB12556DB9202383F306
:101C600011882B462A462946FFF736FE85F3118850
:101C70000A2384F834300EE0142384F8343020230F
:101C800083F3118800231A4619462046FFF712FEF7
:101C9000002383F3118838BD036C03B198470023F8
:101CA000E7E70021204601F051FA0021204601F02B
:101CB00043FA63681B6813B1062120469847062340
:101CC000D7E7000010B590F83430142B044629D023
:101CD00017D8062B05D001D81BB110BD093B022B2C
:101CE000FBD80021204601F031FA0021204601F006
:101CF00023FA63681B6813B1062120469847062320
:101D000019E0152BE9D10B2380F83430202383F31D
:101D1000118800231A461946FFF7DEFD002383F3DE
:101D20001188DAE7C3689B695B68002BD5D1036C27
:101D300003B19847002384F83430CEE7024B0022E9
:101D4000C3E900339A607047202600200023037403
:101D50008268054B1B6899689142FBD25A68036000
:101D600042601060586070472026002008B520238C
:101D700083F31188037C032B05D0042B0DD02BB9E2
:101D800083F3118808BD436900221A604FF0FF33C6
:101D90004361FFF7DBFF0023F2E7D0E90032136075
:101DA0005A60F3E7002303748268054B1B68996847
:101DB0009142FBD85A6803604260106058607047D7
:101DC00020260020054B19690874186802681A60FB
:101DD0005360186101230374FEF798BA202600208F
:101DE00030B54B1C0B4D87B0044610D02B690A4A06
:101DF00001A800F025F92046FFF7E4FF049B13B18A
:101E000001A800F059F92B69586907B030BDFFF7F8
:101E1000D9FFF8E7202600206D1D000838B50C4DCD
:101E200041612B6981689A689142044603D8BDE8F4
:101E30003840FFF78BBF1846FFF7B4FF01232C6132
:101E4000014623742046BDE83840FEF75FBA00BF64
:101E500020260020044B1A681B6990689B689842F2
:101E600094BF0020012070472026002010B5084CA8
:101E7000236820691A6822605460012223611A7461
:101E8000FFF790FF01462069BDE81040FEF73EBA1B
:101E90002026002008B5FFF7DDFF18B1BDE8084097
:101EA000FFF7E4BF08BD0000FFF7E0BFFEE700005A
:101EB00010B50C4CFFF742FF00F0B4F80A4980223D
:101EC000204600F03BF8012344F8180C037400F09E
:101ED00071FC002383F3118862B60448BDE810400A
:101EE00000F04CB848260020583B0008683B00082A
:101EF00000F01CB9EFF3118020B9EFF30583202225
:101F000082F311887047000010B530B9EFF30584F3
:101F1000C4F3080414B180F3118810BDFFF7BAFFB1
:101F200084F31188F9E70000034A516853685B1A8B
:101F30009842FBD8704700BF001000E08260022288
:101F4000028270478368A3F17C0243F80C2C02697B
:101F500043F83C2C426943F8382C074A43F81C2CC0
:101F6000C26843F8102C022203F8082C002203F860
:101F7000072CA3F1180070472503000810B5202393
:101F800083F31188FFF7DEFF00210446FFF746FFC9
:101F9000002383F31188204610BD0000024B1B690B
:101FA00058610F20FFF70EBF20260020202383F367
:101FB0001188FFF7F3BF000008B50146202383F323
:101FC00011880820FFF70CFF002383F3118808BD58
:101FD00049B1064B42681B6918605A601360436040
:101FE0000420FFF7FDBE4FF0FF3070472026002091
:101FF0000368984206D01A6802605060596118461A
:10200000FFF7A4BE7047000038B504460D462068AF
:10201000844200D138BD036823605C604561FFF7EE
:1020200095FEF4E7054B03F11402C3E905224FF0D6
:10203000FF310022C3E90712704700BF20260020AD
:1020400070B51C4EC0E9032305460C4601F07AFA30
:10205000334653F8142F9A420DD13062C5E901245A
:102060002A600A2C2CBF00190A30C6E90555BDE8C4
:10207000704001F055BA316A431AE31838BF1C4664
:102080009368A34202D9081901F058FA73699A6853
:1020900094420CD85A68AC602B606A6015609A68EC
:1020A0005D60121B9A604FF0FF33F36170BD1B68D7
:1020B000A41AECE72026002038B51B4C636998422F
:1020C0000DD0D0E9003213605A6000228168C260EE
:1020D0009A680A449A604FF0FF33E36138BD2246A4
:1020E000036842F8143F002193425A60C16003D153
:1020F000BDE8384001F01CBA9A688168256A0A4434
:102100009A6001F01FFA63699A68411B8A42E5D917
:10211000AB181D1A092D206A98BF01F10A02BDE80B
:102120003840104401F00ABA202600202DE9F04181
:10213000184C002704F11406656901F003FA236ABC
:10214000AA68C11A8A4215D813442362D5E900321D
:1021500013605A606369D5F80C80EF60B34201D117
:1021600001F0E6F987F311882869C047202383F33B
:102170001188E1E76169B14209D013441B1ABDE837
:10218000F0410A2B2CBFC0180A3001F0D7B9BDE8C6
:10219000F08100BF2026002000207047FEE70000ED
:1021A000704700004FF0FF307047000002290CD04C
:1021B000032904D00129074818BF00207047032ACB
:1021C00005D8054800EBC20070470448704700205E
:1021D000704700BF4C3C00082C220020003C000847
:1021E00070B59AB00546084601A9144600F0C2F839
:1021F00001A8FEF78BFD431C5B00C5E900340022FB
:10220000237003236370C6B201AB02341046D1B20F
:102210008E4204F1020401D81AB070BD13F8011BFC
:1022200004F8021C04F8010C0132F0E708B5202381
:1022300083F311880348FFF779FA002383F31188A9
:1022400008BD00BFD827002090F8443003F01F02DB
:10225000012A07D190F845200B2A03D10023C0E9B9
:102260000E3315E003F06003202B08D1B0F848309E
:102270002BB990F84520212A03D81F2A04D8FFF74C
:1022800037BA222AEBD0FAE7034A82630722C263F5
:1022900003640120704700BF2322002007B50529F1
:1022A00017D8DFE801F0191603191920202383F34A
:1022B0001188104A01900121FFF7D8FA01980E4ABF
:1022C0000221FFF7D3FA0D48FFF7FCF9002383F34F
:1022D000118803B05DF804FB202383F311880748BD
:1022E000FFF7C6F9F2E7202383F311880348FFF7CD
:1022F000DDF9EBE7A03B0008C43B0008D82700202D
:1023000038B50C4D0C4C0D492A4604F10800FFF776
:1023100067FF05F1CA0204F110000949FFF760FFE9
:1023200005F5CA7204F118000649BDE83840FFF708
:1023300057BF00BFA02C00202C220020803B0008AB
:102340008A3B0008953B000870B5044608460D46D8
:10235000FEF7DCFCC6B22046013403780BB9184600
:1023600070BD32462946FEF7BDFC0028F3D101209E
:10237000F6E700002DE9F04705460C46FEF7C6FCDF
:102380002B49C6B22846FFF7DFFF08B10736F6B281
:1023900028492846FFF7D8FF08B11036F6B2632E59
:1023A0000BD8DFF88C80DFF88C90234FDFF894A0F7
:1023B0002E7846B92670BDE8F08729462046BDE84C
:1023C000F04701F051BB252E2ED107224146284669
:1023D000FEF788FC70B9194B224603F10C0153F843
:1023E000040B42F8040B8B42F9D11B88138007358C
:1023F0000E34DDE7082249462846FEF773FC98B9FB
:102400000F4BA21C197809090232C95D02F8041C9D
:1024100013F8011B01F00F015345C95D02F8031CBD
:10242000F0D118340835C3E704F8016B0135BFE774
:102430006C3C0008953B0008833C0008743C000895
:10244000107AFF1F1C7AFF1FBFF34F8F024AD36819
:10245000DB03FCD4704700BF003C024008B5094BC9
:102460001B7873B9FFF7F0FF074B1A69002ABFBF4B
:10247000064A5A6002F188325A601A6822F4806271
:102480001A6008BDFE2E0020003C02402301674573
:1024900008B50B4B1B7893B9FFF7D6FF094B1A69A8
:1024A00042F000421A611A6842F480521A601A68B7
:1024B00022F480521A601A6842F480621A6008BDE1
:1024C000FE2E0020003C02400B28F0B516D80C4C24
:1024D0000C4923787BB90C4D0E460C234FF000625B
:1024E00055F8047B46F8042B013B13F0FF033A44F4
:1024F000F6D10123237051F82000F0BD0020FCE745
:10250000302F0020002F0020943C0008014B53F88E
:1025100020007047943C00080C2070470B2810B531
:10252000044601D9002010BDFFF7CEFF064B53F83B
:1025300024301844C21A0BB90120F4E712680132A2
:10254000F0D1043BF6E700BF943C00080B2838B5F7
:10255000044628D8FFF7CEFCFFF776FFFFF77EFF93
:10256000124AF323D360E300DBB243F4007343F079
:1025700002031361136943F4803313610546204657
:10258000FFF762FFFFF7A0FF094B53F8241000F09C
:10259000E9F82846FFF77CFFFFF7B6FC2046BDE8C8
:1025A0003840FFF7BBBF002038BD00BF003C0240F1
:1025B000943C000812F001032DE9F04105460E4657
:1025C00014464BD18218B2F1016F61D8314B1B68B0
:1025D00013F001035CD0304FFFF78CFCFFF73EFF98
:1025E000F323FB60FFF730FF314640F20128032C54
:1025F00018D824F00104284E0C446D1A40F201183A
:10260000A142336905EB01072AD123F001033361AD
:10261000FFF73EFFFFF778FC0120BDE8F081043CA6
:102620000435E4E7AB07E4D13B6923F440733B6135
:102630003B6943EA08033B6151F8046B2E60BFF32A
:102640004F8FFFF701FF2B689E42E8D03B6923F0D4
:1026500001033B61FFF71CFFFFF756FC0020DCE79E
:1026600023F440733361336943EA080333610B8811
:102670003B80BFF34F8FFFF7E7FE3F8831F8023B07
:10268000BFB2BB42BCD0336923F001033361E1E741
:102690001846C2E700380240003C0240084908B52D
:1026A0000B7828B11BB9FFF7D9FE01230B7008BDC9
:1026B000002BFCD0BDE808400870FFF7E9BE00BF62
:1026C000FE2E002010B50244064BD2B2904200D13B
:1026D00010BD441C00B253F8200041F8040BE0B2D6
:1026E000F4E700BF502800400F4B30B51C6F2404A6
:1026F00007D41C6F44F400741C671C6F44F400443E
:102700001C670A4C236843F4807323600244084B1F
:10271000D2B2904200D130BD441C00B251F8045BEB
:1027200043F82050E0B2F4E7003802400070004067
:102730005028004007B5012201A90020FFF7C2FF81
:10274000019803B05DF804FB13B50446FFF7F2FFF0
:10275000A04205D0012201A900200194FFF7C4FF87
:1027600002B010BD70470000034B1A681AB9034A43
:10277000D2F874281A607047342F002000300240CD
:1027800008B5FFF7F1FF024B1868C0F3407008BDB1
:10279000342F0020EFF3098305494A6B22F0010230
:1027A0004A63683383F30988002383F311887047F1
:1027B00000EF00E0202080F3118862B60C4B0D4A38
:1027C000D96821F4E0610904090C0A43DA60D3F8FE
:1027D000FC20094942F08072C3F8FC200A6842F0EC
:1027E00001020A601022DA7783F82200704700BFE6
:1027F00000ED00E00003FA05001000E010B5202312
:1028000083F311880E4B5B6813F4006314D0F1EE70
:10281000103AEFF30984683C4FF08073E361094B91
:10282000DB6B236684F30988FFF714FB10B1064BBA
:10283000A36110BD054BFBE783F31188F9E700BFE7
:1028400000ED00E000EF00E0370300083A03000865
:1028500070470000FEE700000A4B0B480B4A90420D
:102860000BD30B4BDA1C121AC11E22F003028B424F
:1028700038BF00220021FEF751BA53F8041B40F87C
:10288000041BECE73C3E00083030002030300020D4
:10289000303000207047000070B5D0E915439E68C5
:1028A00000224FF0FF3504EB42135101D3F8000929
:1028B0000028BEBFD3F8000940F08040C3F80009EB
:1028C000D3F8000B0028BEBFD3F8000B40F08040C7
:1028D000C3F8000B013263189642C3F80859C3F8D5
:1028E000085BE0D24FF00113C4F81C3870BD000043
:1028F0001D4B03EB80022DE9F043D2F80CC05D6D57
:10290000DCF81420461CD2F800E005EB063605EB97
:102910004018516871450AD3D5F83438012202FABB
:1029200000F023EA0000C5F83408BDE8F083BCF8E5
:102930001040AEEB0103A34228BF2346D8F8184944
:10294000A4B2B3EB840FF0D89468A4F1040959F849
:10295000047F3760A4EB09071F44042FF7D81C44F9
:102960000B4494605360D4E7382F0020890141F074
:102970002001016103699B06FCD41220FFF7D4BA41
:1029800010B5054C2046FEF753FF4FF0A04363659A
:10299000024BA36510BD00BF382F0020E83C0008A3
:1029A00070B50378012B054650D12A4B446D9842EF
:1029B0001BD1294B5A6B42F080025A635A6D42F088
:1029C00080025A655A6D5A6942F080025A615A690A
:1029D00022F080025A610E2143205B69FEF79AFBC8
:1029E0001E4BE3601E4BC4F800380023C4F8003EC1
:1029F000C02323606E6D4FF40413A3633369002B6F
:102A0000FCDA012333610C20FFF78EFA3369DB0710
:102A1000FCD41220FFF788FA3369002BFCDA002679
:102A2000A6602846FFF738FF6B68C4F81068DB68BB
:102A3000C4F81468C4F81C684BB90A4BA3614FF082
:102A4000FF336361A36843F00103A36070BD064BCD
:102A5000F4E700BF382F0020003802404014004047
:102A600003002002003C30C0083C30C0F8B5446D83
:102A7000054600212046FFF779FFA96D00234FF09E
:102A800001128F68C4F834384FF00066C4F81C286F
:102A90004FF0FF3004EB431201339F42C2F800694C
:102AA000C2F8006BC2F80809C2F8080BF2D20B6832
:102AB0006A6DEB65636210231361166916F01006E8
:102AC000FBD11220FFF730FAD4F8003823F4FE636C
:102AD000C4F80038A36943F4402343F01003A36112
:102AE0000923C4F81038C4F814380A4BEB604FF0CF
:102AF000C043C4F8103B084BC4F8003BC4F810694D
:102B0000C4F80039EB6D03F1100243F48013EA6559
:102B1000A362F8BDC43C000840800010426D90F8EC
:102B20004E10D2F8003823F4FE6343EA0113C2F8D2
:102B3000003870472DE9F84300EB8103456DDA68F2
:102B4000166806F00306731E022B05EB41130C46B4
:102B500080460FFA81F94FEA41104FF00001C3F8A7
:102B6000101B4FF0010104F1100398BFB60401FAE5
:102B700003F391698EBF334E06F1805606F5004689
:102B800000293AD0578A04F15801490137436F5060
:102B9000D5F81C180B43C5F81C382B180021C3F8B6
:102BA000101953690127611EA7409BB3138A928BAA
:102BB0009B08012A88BF5343D8F85C20981842EA42
:102BC000034301F1400205EB8202C8F85C00214694
:102BD00053602846FFF7CAFE08EB8900C3681B8ACA
:102BE00043EA8453483464011E432E51D5F81C38FF
:102BF0001F43C5F81C78BDE8F88305EB4917D7F8E3
:102C0000001B21F40041C7F8001BD5F81C1821EA6D
:102C10000303C0E704F13F0305EB83030A4A5A604C
:102C200028462146FFF7A2FE05EB4910D0F80039EF
:102C300023F40043C0F80039D5F81C3823EA07070D
:102C4000D7E700BF0080001000040002826D126808
:102C5000C265FFF721BE00005831436D49015B5842
:102C600013F4004004D013F4001F0CBF0220012015
:102C7000704700004831436D49015B5813F4004030
:102C800004D013F4001F0CBF022001207047000085
:102C900000EB8101CB68196A0B6813604B685360C5
:102CA0007047000000EB810330B5DD68AA69136846
:102CB000D36019B9402B84BF402313606B8A14681A
:102CC000426D1C44013CB4FBF3F46343033323F033
:102CD000030302EB411043EAC44343F0C043C0F88E
:102CE000103B2B6803F00303012B09B20ED1D2F87D
:102CF000083802EB411013F4807FD0F8003B14BF7A
:102D000043F0805343F00053C0F8003B02EB411204
:102D1000D2F8003B43F00443C2F8003B30BD000052
:102D20002DE9F041244D6E6D06EB40130446D3F8B7
:102D3000087BC3F8087B38070AD5D6F8143819077A
:102D400006D505EB84032146DB6828465B68984777
:102D5000FA071FD5D6F81438DB071BD505EB84031B
:102D6000D968CCB98B69488A5A68B2FBF0F600FB87
:102D700016228AB91868DA6890420DD2121AC3E98D
:102D80000024202383F311880B482146FFF78AFF94
:102D900084F31188BDE8F081012303FA04F26B8902
:102DA00023EA02036B81CB68002BF3D02146024853
:102DB000BDE8F041184700BF382F002000EB810329
:102DC00070B5DD68436D6C692668E6604A0156BBE4
:102DD0001A444FF40020C2F810092A6802F00302D6
:102DE000012A0AB20ED1D3F8080803EB421410F4FA
:102DF000807FD4F8000914BF40F0805040F00050AC
:102E0000C4F8000903EB4212D2F8000940F0044074
:102E1000C2F80009D3F83408012202FA01F1014393
:102E2000C3F8341870BD19B9402E84BF402020600B
:102E300020682E8A8419013CB4FBF6F440EAC440B1
:102E400040F000501A44C6E7F8B504461E48456DE8
:102E500005EB4413D3F80869C3F80869F10717D5DF
:102E6000D5F81038DA0713D500EB8403D9684B691D
:102E70001F68DA68974218D2D21B00271A605F6079
:102E8000202383F311882146FFF798FF87F31188E9
:102E9000330617D5D5F834280123A340134211D0A7
:102EA0002046BDE8F840FFF723BD012303FA04F2F2
:102EB000038923EA020303818B68002BE8D02146B3
:102EC0009847E5E7F8BD00BF382F00202DE9F74F00
:102ED000984C666D7569B3691D4015F4805875612D
:102EE00007D02046FEF70AFD03B0BDE8F04FFFF71C
:102EF00085BC002D12DAD6F8003E8E489F071EBF13
:102F0000D6F8003E23F00303C6F8003ED6F8043896
:102F100023F00103C6F80438FEF718FD280505D58F
:102F20008448FFF7B9FC8348FEF700FDA9040CD5DF
:102F3000D6F8083813F0060FF36823F470530CBF6B
:102F400043F4105343F4A053F3602A0704D5636895
:102F5000DB680BB177489847EB0274D4AF0227D5F2
:102F6000D4F85490DFF8CCB100274FF0010A09EBF8
:102F70004712D2F8003B03F44023B3F5802F11D160
:102F8000D2F8003B002B0DDA62890AFA07F322EA35
:102F90000303638104EB8703DB68DB6813B1394605
:102FA00058469847A36D01379B68FFB29F42DED910
:102FB000E80617D5676D3A6AC2F30A1002F00F03EC
:102FC00002F4F012B2F5802F00F08880B2F5402FA5
:102FD00008D104EB83030022DB681B6A07F58057E6
:102FE00090426DD12903D6F8184813D5E20302D5D3
:102FF0000020FFF795FEA30302D50120FFF790FE06
:10300000670302D50220FFF78BFE260302D50320BB
:10301000FFF786FE6D037FF567AFE00702D500205E
:10302000FFF712FFA10702D50120FFF70DFF62078E
:1030300002D50220FFF708FF23077FF555AF0320D5
:10304000FFF702FF50E7636DDFF8E8B00193002758
:103050004FF0010AA36D9B685FFA87F999453FF627
:103060007DAF019B03EB4913D3F8002902F4402202
:10307000B2F5802F22D1D3F80029002A1EDAD3F826
:10308000002942F09042C3F80029D3F80029002A11
:10309000FBDB606D4946FFF769FC22890AFA09F3F8
:1030A00022EA0303238104EB8903DB689B6813B1E5
:1030B0004946584698474846FFF71AFC0137C9E782
:1030C000910708BFD7F80080072A98BF03F8018B43
:1030D00002F1010298BF4FEA182881E7023304EB9E
:1030E000830207F580575268D2F818C0DCF8082030
:1030F000DCE9001CA1EB0C0C002188420AD104EB96
:10310000830463689B699A6802449A605A6802441F
:103110005A6067E711F0030F08BFD7F800808C45AD
:1031200088BF02F8018B01F1010188BF4FEA18281E
:10313000E3E700BF382F0020436D03EB4111D1F8C6
:10314000003B43F40013C1F8003B7047436D03EBB1
:103150004111D1F8003943F40013C1F80039704728
:10316000436D03EB4111D1F8003B23F40013C1F888
:10317000003B7047436D03EB4111D1F8003923F454
:103180000013C1F80039704730B5039C0172043355
:1031900004FB0325C0E90653049B03630021059B40
:1031A000C160C0E90000C0E90422C0E90842C0E9EA
:1031B0000A11436330BD0000416A0022C0E90411D6
:1031C000C0E90A22C2606FF00101FEF71DBF0000D6
:1031D000D0E90432934201D1C2680AB9181D704780
:1031E0000020704703691960C2680132C260C26979
:1031F000134482690361934224BF436A036100213F
:10320000FEF7F6BE38B504460D46E3683BB1626989
:10321000131D1268A3621344E362002007E0237ABF
:1032200033B929462046FEF7D3FE0028EDDA38BD33
:103230006FF00100FBE70000C368C269013BC36097
:103240004369134482694361934224BF436A4361E3
:1032500000238362036B03B11847704770B52023C6
:10326000044683F31188866A3EB9FFF7CBFF054613
:1032700018B186F31188284670BDA36AE26A13F874
:10328000015BA362934202D32046FFF7D5FF0023E0
:1032900083F31188EFE700002DE9F84F04460E464E
:1032A000174698464FF0200989F311880025AA4651
:1032B000D4F828B0BBF1000F09D141462046FFF7F2
:1032C000A1FF20B18BF311882846BDE8F88FD4E91F
:1032D0000A12A7EB050B521A934528BF9346BBF180
:1032E000400F1BD9334601F1400251F8040B43F85B
:1032F000040B9142F9D1A36A40334036A3624035B2
:10330000D4E90A239A4202D32046FFF795FF8AF3B5
:103310001188BD42D8D289F31188C9E730465A4690
:10332000FDF7D6FCA36A5B445E44A3625D44E7E715
:1033300010B5029C0172043304FB0321C0E906139B
:103340000023C0E90A33039B0363049BC460C0E904
:103350000000C0E90422C0E90842436310BD000038
:10336000026AC260426AC0E904220022C0E90A225D
:103370006FF00101FEF748BED0E904239A4201D163
:10338000C26822B9184650F8043B0B607047002011
:1033900070470000C368C2690133C36043691344C6
:1033A00082694361934224BF436A43610021FEF76F
:1033B0001FBE000038B504460D46E3683BB12369E3
:1033C0001A1DA262E2691344E362002007E0237A37
:1033D00033B929462046FEF7FBFD0028EDDA38BD5B
:1033E0006FF00100FBE7000003691960C268013A51
:1033F000C260C269134482690361934224BF436A75
:10340000036100238362036B03B118477047000018
:1034100070B520230D460446114683F31188866A51
:103420002EB9FFF7C7FF10B186F3118870BDA36AEC
:103430001D70A36AE26A01339342A36204D3E16977
:1034400020460439FFF7D0FF002080F31188EDE714
:103450002DE9F84F04460D46904699464FF0200A54
:103460008AF311880026B346A76A4FB94946204619
:10347000FFF7A0FF20B187F311883046BDE8F88F31
:10348000D4E90A073A1AA8EB0607974228BF17465D
:10349000402F1BD905F1400355F8042B40F8042BAD
:1034A0009D42F9D1A36A4033A3624036D4E90A238E
:1034B0009A4204D3E16920460439FFF795FF8BF364
:1034C00011884645D9D28AF31188CDE729463A4674
:1034D000FDF7FEFBA36A3B443D44A3623E44E5E79F
:1034E000D0E904239A4217D1C3689BB1836A8BB198
:1034F000043B9B1A0ED01360C368013BC360C369D1
:103500001A44836902619A4224BF436A036100231B
:1035100083620123184670470023FBE700F088B858
:103520004FF08043002258631A610222DA6070472C
:103530004FF080430022DA60704700004FF0804374
:10354000586370474FF08043586A70474B68436038
:103550008B688360CB68C3600B6943614B6903620E
:103560008B6943620B6803607047000008B5264B07
:1035700026481A6940F2FF110A431A611A6922F4B7
:10358000FF7222F001021A611A691A6B0A431A6368
:103590001A6D0A431A651E4A1B6D1146FFF7D6FFC6
:1035A00002F11C0100F58060FFF7D0FF02F1380145
:1035B00000F58060FFF7CAFF02F1540100F580605A
:1035C000FFF7C4FF02F1700100F58060FFF7BEFF56
:1035D00002F18C0100F58060FFF7B8FF02F1A8014D
:1035E00000F58060FFF7B2FF02F1C40100F58060D2
:1035F000FFF7ACFF02F1E00100F58060FFF7A6FFE6
:10360000BDE8084000F09AB80038024000000240CF
:10361000F43C000808B500F007FAFEF749FCFFF794
:10362000A3F8BDE80840FEF76BBE0000704700003D
:10363000104B1A6C42F001021A641A6E42F0010239
:103640001A660D4A1B6E936843F0010393604FF0B6
:10365000804353229A624FF0FF32DA6200229A616D
:103660005A63DA605A6001225A6108211A601C20EC
:10367000FDF750BD00380240002004E04FF08042CA
:1036800008B51169D3680B40D9B2C9439B071161D2
:1036900007D5202383F31188FEF72AFC002383F348
:1036A000118808BD08B5FFF7E9FFBDE80840FFF73E
:1036B000A5B800001F4B1A696FEAC2526FEAD252D6
:1036C0001A611A69C2F308021A614FF0FF301A69D1
:1036D0005A69586100215A6959615A691A6A62F037
:1036E00080521A621A6A02F080521A621A6A5A6A80
:1036F00058625A6A59625A6A1A6C42F080521A64C5
:103700001A6E42F080521A661A6E0B4A106840F424
:1037100080701060186F00F44070B0F5007F1EBF1D
:103720004FF4803018671967536823F400735360AF
:1037300000F05AB90038024000700040334B4FF09F
:1037400080521A64324A4FF4404111601A6842F0C4
:1037500001021A601A689107FCD59A6822F00302E8
:103760009A602A4B9A6812F00C02FBD1196801F09A
:10377000F90119609A601A6842F480321A601A6876
:103780009203FCD55A6F42F001025A671F4B5A6FE1
:103790009007FCD51F4A5A601A6842F080721A607E
:1037A0001B4A53685904FCD5184B1A689201FCD582
:1037B000194A9A60194B1A68194B9A42194B21D130
:1037C000194A1168194A91421CD140F205121A6037
:1037D000144A136803F00F03052BFAD10B4B9A68B8
:1037E00042F002029A609A6802F00C02082AFAD1AA
:1037F0005A6C42F480425A645A6E42F480425A66CD
:103800005B6E704740F20572E1E700BF003802408E
:10381000007000400854400700948838002004E0FD
:1038200011640020003C024000ED00E041C20F4165
:10383000084A08B5516913680B4003F0010353614E
:1038400023B1054A13680BB150689847BDE808409A
:10385000FEF7D4BF003C0140B02F0020084A08B555
:10386000516913680B4003F00203536123B1054A09
:1038700093680BB1D0689847BDE80840FEF7BEBF1B
:10388000003C0140B02F0020084A08B55169136878
:103890000B4003F00403536123B1054A13690BB1D4
:1038A00050699847BDE80840FEF7A8BF003C0140BA
:1038B000B02F0020084A08B5516913680B4003F087
:1038C0000803536123B1054A93690BB1D069984746
:1038D000BDE80840FEF792BF003C0140B02F002039
:1038E000084A08B5516913680B4003F0100353618F
:1038F00023B1054A136A0BB1506A9847BDE80840E6
:10390000FEF77CBF003C0140B02F0020174B10B5E4
:103910005A691C68144004F478725A61A30604D5ED
:10392000134A936A0BB1D06A9847600604D5104ACF
:10393000136B0BB1506B9847210604D50C4A936B5F
:103940000BB1D06B9847E20504D5094A136C0BB153
:10395000506C9847A30504D5054A936C0BB1D06C05
:103960009847BDE81040FEF749BF00BF003C01404A
:10397000B02F00201A4B10B55A691C68144004F48B
:103980007C425A61620504D5164A136D0BB1506D25
:103990009847230504D5134A936D0BB1D06D984712
:1039A000E00404D50F4A136E0BB1506E9847A10482
:1039B00004D50C4A936E0BB1D06E9847620404D5BF
:1039C000084A136F0BB1506F9847230404D5054A7A
:1039D000936F0BB1D06F9847BDE81040FEF70EBF54
:1039E000003C0140B02F0020062108B50846FDF735
:1039F00091FB06210720FDF78DFB06210820FDF72E
:103A000089FB06210920FDF785FB06210A20FDF729
:103A100081FB06211720FDF77DFBBDE8084006214C
:103A20002820FDF777BB000008B5FFF743FE00F044
:103A30000DF8FDF713FDFDF7F9FEFDF7D1FDFFF7DA
:103A4000F5FDBDE80840FFF769BD00000023054A09
:103A500019460133102BC2E9001102F10802F8D116
:103A6000704700BFB02F0020034611F8012B03F868
:103A7000012B002AF9D1704753544D3332463F3F52
:103A80003F00000053544D333246343078005354D5
:103A90004D3332463432780053544D333246343449
:103AA00036585800012033000010410001105A0020
:103AB000031059000710310000000000783A000898
:103AC0003F00000013040000843A00083F0000009B
:103AD000190400008E3A00083F0000002104000095
:103AE000983A00083F000000009600000000000027
:103AF00000000000000000000000000000000000C6
:103B000025140008111400084D1400083914000889
:103B100045140008311400081D1400080914000899
:103B200059140008000000005D1500084915000840
:103B300085150008711500087D1500086915000835
:103B400055150008411500089115000800000000F7
:103B500001000000000000006D61696E00000000BF
:103B600069646C6500000000603B0008602600206E
:103B7000D827002001000000AD1E00080000000052
:103B80004172647550696C6F740025424F41524414
:103B9000252D424C002553455249414C250000003B
:103BA000020000000000000079170008E517000877
:103BB00040004000702C0020802C002002000000FB
:103BC00000000000030000000000000029180008A9
:103BD0000000000010000000902C002000000000F9
:103BE0000100000000000000382F00200101020049
:103BF0009D220008AD210008492200082D2200085E
:103C000043000000083C000809024300020100C014
:103C10003209040000010202010005240010010520
:103C20002401000104240202052406000107058284
:103C3000030800FF09040100020A00000007050153
:103C40000240000007058102400000001200000051
:103C5000543C0008120110010200004009124157B3
:103C600000020102030100000403090425424F4140
:103C7000524425004D6174656B463430352D5654E1
:103C80004F4C0030313233343536373839414243C6
:103C90004445460000400000004000000040000095
:103CA00000400000000001000000020000000200CF
:103CB00000000200000002000000020000000200FC
:103CC000000002000000000061190008191C000833
:103CD000C51C000840004000982F0020982F0020AD
:103CE00001000000A82F002080000000400100001B
:103CF000030000000001A81600000000AAAAAAAA5A
:103D000000001400EF9F00000000000070A70A00F0
:103D10000004000100000000AAAAAAAA00000001F5
:103D2000DFFF00000000000000000000040000149D
:103D300000000000AAAAAAAA04000014FFFF0000C5
:103D40000000000000000000000000000000000073
:103D5000AAAAAAAA00000000FFFF000000000000BD
:103D6000000000000000000000000000AAAAAAAAAB
:103D700000000000FFFF0000000000000000000045
:103D80000000000000000000AAAAAAAA000000008B
:103D9000FFFF000000000000000000000000000025
:103DA00000000000AAAAAAAA00000000FFFF00006D
:103DB0000000000000000000000000000000000003
:103DC0000A000000000000000300000000000000E6
:103DD00000000000000000000000000000000000E3
:103DE00000000000000000000000000000000000D3
:103DF0001E0400000000000000000F000000000092
:103E0000FF000000D8270020B82300200096000003
:103E100000000800960000000008000004000000F8
:103E2000683C0008000000000000000000000000E6
:0C3E300000000000000000000000000086
:00000001FF
